:020000020000FC
:100000000C94B40FE8C100000000000000000000E4
:1000100000000000000000000000000000000000E0
:10002000000000002EC00000000000009EC0000084
:1000300000000000000000000000000000000000C0
:10004000A7C0000000000000000000000000000049
:100050000000000002030406080C10182030406065
:1000600080000406080C10182030406080A0C000FA
:1000700000070F1F3F000D0D0403060D05020302CC
:1000800002004FB662FD0FC0552009F00994C52D3E
:10009000C095089483FDC795C093B200C0934101F9
:1000A00064604FBE1895C0910401089483FDC79504
:1000B000C093B200C09341016B7FC0910401CF3F58
:1000C00009F41BC04FBE2B982C982D9818952B988F
:1000D0002C982D9875FD0DC065FD0BC0C5E0CA9527
:1000E000F1F7C0915301C0FD2A9AC1FD289AC2FDC3
:1000F000299A209241014FBE18952092B200CC2738
:10010000C160C7BB6460F5CFC2CF70FFC0CF65FDD3
:10011000BECF2B9ABCCF70FFBACF65FDB8CF2C9A5B
:10012000B6CF70FFB4CF65FDB2CF2D9AB0CF2A986D
:1001300070FFADCF65FDABCFC1E4CA95F1F72B9A47
:10014000A6CF289870FFA3CF65FDA1CFC1E4CA95C3
:10015000F1F72C9A9CCF299870FF99CF65FD97CF26
:10016000C1E4CA95F1F72D9A92CF4FB6C0916F00B6
:10017000CD7FC0936F006E7FC0918400CE0DD09173
:100180008500DF1DD0938900C09388004FBE18956D
:100190003FB68F7EADB3A170A2118061A0E0ADBB70
:1001A000A0916E00AE7FA0936E007894A09108019C
:1001B000AA2341F085FD2BC0A0910801AA95A09328
:1001C000080125C040E050E085FD15C0A9B196FDAD
:1001D000A095A2FD4FEFA3E096FDA2E0A0936900D9
:1001E000AA27A160ACBB8D7FA9B196FDA095A2FD09
:1001F0005FEF451739F7A0E461FDA093080185FD85
:1002000003C0A0E4A093080140933701816085FDFD
:100210000EC0A0910901AA2331F0A0910901AA956D
:10022000A093090104C08061AA27A160ACBB80FF34
:100230000AC0A09137014A2F61FF8E7F85FD01C062
:1002400000C04093010140915601443009F004C0C0
:10025000A0910101A0930301A52DA03408F06860CE
:10026000A0910001A395A093000161F0F894A091E2
:100270006E00A160A0936E0084FF02C0A1E0ADBB40
:100280003FBE1895A0911401A395A093140142E0DC
:1002900050910801552329F085FF03C05A955093CA
:1002A0000801A0913701A13018F020923A010DC049
:1002B00020923B0120924501A0913A01AF5FA093AB
:1002C0003A0118F0AFEFA0933A01B09001015091BC
:1002D0005601523049F466FF91F0A2E3BA1678F065
:1002E000A0912701A0930101533049F466FF39F032
:1002F000A2E3BA1620F0A0916201A09301015091EF
:1003000002015B1521F010F05A9501C053955093EE
:1003100002014A95D1F650914501539509F45A9539
:1003200050934501A0914601AA95A093460109F07A
:1003300046C0A1E0A093460145E0A09147015A17AD
:10034000F0F1A09148015A1728F441E0A3E0A093EE
:10035000460107C0A09149015A1718F441E04093A3
:100360004601D0903D01C0900301DC14A8F0A0919B
:100370005601A430D9F066FD0FC0C0923D015395DF
:1003800011F0A0914701A0934501A1E0A09346017F
:10039000ACE3A093020113C0A0913D01A40F20F48F
:1003A0005FEF50933D0102C0A0933D01A0913D013C
:1003B000AF3F29F4AFEFA0933B01A0934501F89420
:1003C000A0916E00A160A0936E0084FF02C0A1E026
:1003D000ADBB3FBE18953FB640918400509185005B
:1003E0008F7EADB3A170A2118061A0E0ADBBA091E2
:1003F0006E00AE7FA0936E00789481FD25C0A2E0D0
:1004000096FDA3E0A09369008260A9B196FDA09536
:10041000A2FF05C040930501509306011FC1A3E050
:1004200096FDA2E0A0936900AA27A160ACBB8D7FD6
:1004300085FF01C006C140E0A9B196FDA095A2FDCF
:1004400000C140933701EFC0A3E096FDA2E0A09366
:1004500069008D7F61FF72C0A2E096FDA3E0A093CA
:100460006900AA27A160ACBB82604093320150931F
:100470003301A09030014A19B09031015B09BB24CF
:10048000A22C4C38520518F42092360149C0A09194
:100490007601AA2359F1483C520528F4A0E1BA2E6E
:1004A000AAE0AA2E23C04836A1E05A0728F4A8E003
:1004B000BA2EAFE0AA2E1AC0403DA2E05A0728F497
:1004C000A4E0BA2EAEE1AA2E11C0403AA5E05A0728
:1004D00028F4A2E0BA2EACE3AA2E08C04839A8E05E
:1004E0005A0720F4A1E0BA2EA8E7AA2EC42EA091A4
:1004F0003401CA1AD52EA0913501DA0ADD202AF47A
:10050000AFEFC094D094CA1ADA0A20923601A8E05C
:10051000A210A0E0CA14DA0618F4A1E0A0933601F4
:100520004093340150933501409132015091330191
:10053000409330015093310102E075C0A091050154
:100540004A1BA09106015A0B94FD60C093FD5EC04A
:1005500092FD5AC086FF03C0D52EC42E0CC05695FE
:10056000479591FD51C05695479590FD4DC0D52EAC
:10057000C42ED694C79461FD19C0AC2DAC51AD2DDD
:10058000A24008F005C0DD2089F4AC2DA85C70F411
:10059000A0910701A395AA2311F0A0930701AA3007
:1005A00008F44FC02092370181604BC0A091070131
:1005B000AA2319F0AA95A0930701A22C50915C01DF
:1005C00097FD02C0A0906A01AAEFAA0EA22DA21D5B
:1005D000CA18DA0A4FB74170442319F040E050E0DE
:1005E00015C0AFEFCA16D20418F04FEF50E00EC09E
:1005F000A0914E01CA9E412D000C441F50E008F00E
:1006000012C04FEF50E00FC05695479594FF07C0BA
:10061000552309F04FEFA42FA6954A0F521D4F3FC7
:10062000520508F04FEF40933701816061FF09C028
:10063000AFE1A095A923AB299A2F8F7DBB2009F4A8
:100640008062A0E4A093080185FF03C0AAE0A09304
:10065000080161FD03C085FD01C08F7E85FD03C0DB
:10066000A0E2A0930901F894A0916E00A160A0936C
:100670006E0084FF02C0A1E0ADBB3FBE189511E043
:100680000AC013E008C01AE006C01EE104C014E668
:1006900002C018EC00C005E1BB27BA95F1F70A9536
:1006A000D9F71A95C1F708952AE338E709C020E37E
:1006B0003CE806C02AE234EB03C025E238EC00C077
:1006C00012E095FD9F7D95FF9062BB272898BA9513
:1006D000F1F72C9ABA95F1F72C98BA95F1F7289A78
:1006E000BA95F1F72B9AB0914F01BA95F1F72B9883
:1006F000B7E8BA95F1F71A9521F7022FB22FBA95FC
:10070000F1F70A95D9F73A95D9F628980895221B5A
:1007100039E0001F3A9509F40895221F211B18F4AF
:10072000210F8894F6CF0894F4CF622C722CB0E09D
:100730008894B395221F331FE0F737952795889447
:10074000912E802E020B130B10F4192D082D10F48E
:10075000889401C00894661C771CBA9571F7172D10
:10076000062D0895322D11232AF43A9500951095FF
:10077000031B130BF894029F712C002D129F912CD8
:10078000802C7894780C172D921C292DB4E06B2EB8
:100790002695179507956A94D9F7332321F000958C
:1007A0001095031B130B089500915601043009F4B2
:1007B00074C0B0913701B95198F0B72FB67081F479
:1007C00066FD2BC005E090906801B92DBA9521F027
:1007D0000AE0BA9509F002E1B0911B01B01BE0F00C
:1007E00066FF0AC0B0913F01B0933D01BFEFB093E7
:1007F0004501B1E0B0934601B0910101B09303010E
:1008000020921F012092200120922101209222019A
:10081000209223016F7B41C0606490906801B92DE4
:10082000BA9579F4B0910201B095BB1FBB1F1B2F85
:10083000B7950B2FB12FB170B3951B2FB02FBE7F83
:1008400025C0B92DBA95BA9581F4B0910201B09541
:10085000BB1FBB1FBB1F1B2FB7950B2FB12FB37037
:10086000B3951B2FB02FBC7F14C0B0910201B0957F
:10087000BB1FBB1FBB1FBB1F1B2FB7950B2FB12F60
:10088000B770B395B3951B2FB02FB87FB0540B2F13
:10089000120900931F0110932001089510911B016C
:1008A000169500911A010795B0911F01B01B0B2FEF
:1008B000B0912001B10B1B2F28F40038BFEF1B07AC
:1008C00040F009C00F37120508F405C00FE710E02B
:1008D00002C000E81FEF0093240110932501089542
:1008E00000912401B09121010B0F10912501B091CD
:1008F00022011B1F20E03091250133230AF42A95A1
:10090000B09123012B1F1AF4203F40F00AC02F3072
:1009100008F407C00FEF1FEF2FE003C000E010E066
:1009200020EF30910301B0913C013B1718F43230B5
:1009300030F009C0B0912501BB235AF004C0B0913A
:100940002501BB2332F4009321011093220120934F
:10095000230108952091780100912401000F109146
:100960002501111F0E94B20311232AF40038BFEFA2
:100970001B0740F009C00F37120508F405C00FE748
:1009800010E002C000E81FEF002352F0B091020116
:10099000B01B0B2F18F0013008F00AC001E008C0AE
:1009A00000950F5FB09102010B0F08F001C00FEF2F
:1009B0000093260108952091790100912201109160
:1009C00023010E94B20311232AF40130BFEF1B0759
:1009D00040F009C00F3F120508F405C00FEF10E00A
:1009E00002C001E01FEF112352F0B0912601B01BAD
:1009F0000B2F18F0013008F00AC001E008C0009584
:100A00000F5FB09126010B0F08F001C00FEF0093AC
:100A1000030108950FEF677F71FD2AC072FD09C0C1
:100A20006860B0911B01BA3020F0B52DB03408F4E5
:100A3000677FB0917501BB23D9F0B0911B01BB2337
:100A4000B9F00FEF10911B010E948703F894B09149
:100A5000130172FDB5E00B9F112D002D7894112329
:100A600009F00FEFB0913F010B1710F400913F0117
:100A700000933E01089500911A0110911B0100544A
:100A80001140B0913E0110F4BA9501C0B39511F038
:100A9000B0933E0108950E947609B0E073FDB0E086
:100AA000B06CB0937C00B0917A00B068B064B09341
:100AB0007A000E943F03B0E073FDB0E0B06CB093E9
:100AC0007C00B0917A00B068B064B0937A00B091C5
:100AD0007A00B6FDFCCF0091780010917900B091BA
:100AE0007A00BF77B0937A000E94C70927EE20935F
:100AF0004A01222309F441C030E030934B01732EA8
:100B00007694622E6694620E731E262D372D021780
:100B1000130778F080904A01B7EEB80DB0934A0100
:100B200080904B01B0E0B81DB0934B01260D371DEE
:100B3000EECF80904A0190904B0110914B01169599
:100B400000914A0107951695079523E0169507959C
:100B50002A95E1F7209157012A9529F420924A011C
:100B600020924B010AC02A9521F0800E911E2A95F1
:100B7000E1F780924A0190924B010895209157012C
:100B8000B0917A00B6FDFACF00917800109179000B
:100B9000B0917A00BF77B0937A00B0914C01B395D1
:100BA000B0934C01B83060F120924C01B0917401C7
:100BB000BB2321F1112329F0B0914D01BF3F61F01A
:100BC00009C0B0914D010B1739F020F4BB2321F07F
:100BD000BA9502C0B395E1F300913C01B0934D0189
:100BE000B03050F400ECB03038F400E8B03020F40D
:100BF00000E4B03008F400E000933C01777F0895F2
:100C00002130B1F00F3FB3E01B0790F4B7EEBB23E8
:100C100079F0B0914A010B17B0914B011B0740F4DA
:100C2000B0913C01BB2359F0BA95B0933C0107C089
:100C3000B0913C01BF3F19F0B395B0933C010091D6
:100C40003C01B0910301B01B10F400910301B0917D
:100C50003D010B1750F000913D01B0913D01BF3FA8
:100C600021F0B0913D01B0933C01502E009304015E
:100C7000B0914C01B73009F47860089502E3F8941C
:100C8000B0917A010B9F012D000C001F7894B09158
:100C90003C010B1710F000913C01009301010093FF
:100CA0000301502E0093040100933F010895209208
:100CB0001A01B0EFB0931B010895F89400918400DD
:100CC0001091850020911401789430911501609065
:100CD00016010093150110931601031B160971FDEF
:100CE00003C076FD81C02BC07090170120931701BF
:100CF0002709222311F00FEF1FEF80901801909029
:100D0000190130931801609219016918161910938E
:100D10001C01009115011091160108191909209163
:100D20001A0130911B0136952795020F131F10F4FD
:100D30000FEF1FEF00931A0110931B0129C02091A0
:100D40001A0130911B013901B4E08B2EB2E09B2EC9
:100D5000343010F08A949A94383010F08A949A942F
:100D6000769467948A94E1F726193709992021F03F
:100D7000169507959A94E1F7200F311F20931A01D9
:100D800030931B0128F43FEF30931A0130931B017D
:100D9000323008F4706471FF02C0B3E00DC0B0914E
:100DA000660100911101023838F0B395003A08F05D
:100DB000B395B63008F0B5E09B2EB4E08B2E1091C1
:100DC0001B0100911A0124E0169507952A95E1F779
:100DD0000819120928F0B02FB250B12FB20910F43F
:100DE00002E010E0980126C020911A0130911B0109
:100DF000390176946794669466946694261932094C
:100E000006950695200F321D20931A0130931B0181
:100E1000323008F07F7B04E036952795369527958C
:100E200026952695201B10F0223008F422E0890137
:100E30009090660160FDFECFE0902C01F0902D01B6
:100E40006160B0916F00B260B0936F00380176FDC1
:100E500044C07694679400932C0110932D01B92D12
:100E6000B330E1F0B0FD04C0060D171D930106C0BC
:100E7000000F111F0250120922E030E0B92DB330EB
:100E800068F020932E0130932F01009328011093D6
:100E9000290160922A0170922B013DC000932E011E
:100EA00010932F01209328013093290160922A0189
:100EB00070922B0171FF10C0B0910D01B33060F042
:100EC00000912F0110911C011595010F28F022F0BF
:100ED00020922E0100932F011EC0669400932C01D6
:100EE000B92DB33091F0B0FD03C0060D262D03C01F
:100EF000000F025022E0B92DB33038F020932E01BC
:100F00000093280160922A0106C000932E012093CD
:100F1000280160922A0100911D0102FD0350013059
:100F200039F495FD0EC0B5E0B06CB0937C000DC0F7
:100F3000023029F4B4E0B06CB0937C0006C095FD9B
:100F4000F2CFB3E0B06CB0937C0000914401000F8D
:100F500010F4BBE60B270093440160FDFECFB2E026
:100F6000B0930E016160B0916F00B260B0936F00FA
:100F7000B72FB670D1F020911A0130911B01369530
:100F80002795F8940091840010918500020F131F9B
:100F900010938900009388006160B2E0B6BBB09105
:100FA0006F00B260B0936F007894089560612092F2
:100FB0001E0120E067FD20E206C0606120921E0154
:100FC00020E267FD20E0789401E076FD11C0B72FA4
:100FD000B67009F06F7EB0911B01B55048F002E089
:100FE000B55020F003E0B55008F006E071FD0AE0CE
:100FF00060FD13C0B0911E01BB2379F071FF08C0E2
:10100000B0910D01B33020F0B0910E01BA9519F4F2
:101010007894706168C00E94B20778940000000064
:10102000F89476FD17C010911B01173008F017E0F7
:10103000B5E01B0F72FD10E183FF110F62FF110F6E
:1010400071FD12E8B091B20060904101B61980F2D2
:10105000B10B70F2B0917B00BF7BB0937B00B0B757
:10106000B0917B00B064B0937B00B0911E01B3954A
:10107000B0931E01B0B776FD06C0B1E071FDB2E0DD
:10108000BA95F1F7B0B7B072B21709F021C071FF8D
:1010900005C003950A3008F00395AACF64FF93CFEB
:1010A0006F7E309184006090850070901A0180906E
:1010B0001B01370D681C60928900309388006160C5
:1010C000B2E0B6BBB0916F00B260B0936F007BCF5F
:1010D000B0910D01B23008F476CF64FD74CF0A955B
:1010E00009F086CF7F7E20912E0130912F01F89458
:1010F000B2E0B6BB0091840010918500020F131F6F
:101100001093890000938800E0902801F090290155
:101110006160B0916F00B260B0936F007894B72FA8
:10112000B67039F0B0910D0172FFB395B0930D0117
:1011300009C074FF07C067FD05C064FD03C0BF910F
:10114000BF9178C5089500E063FF03C064FF01C04C
:1011500001E0F89410911101B7E01B9F212D102D93
:101160007894200F2695179526951795269517950F
:1011700010931101183718F4B8E7B09311010091DA
:101180001101B09112010B1720F060622B982C987E
:101190002D9860FDFECFE0902A01F0902B01616058
:1011A000B0916F00B260B0936F000895B2E095FD0A
:1011B00007C0F894B0931D0128982A9A7894E5C046
:1011C000F894B0931D012898299A7894DEC0B3E072
:1011D00082FF24C095FD11C002E0F894B0931D0178
:1011E000E1EAF0E0009353012D98299862FF02C0D4
:1011F0002C9A01C0289A7894C8C002E0F894B09361
:101200001D01E1EAF0E0009353012B982A9862FF58
:1012100002C02C9A01C0289A7894B7C095FD0BC0E3
:10122000F894B0931D01EBE8F0E02D9862FF01C047
:101230002C9A7894AAC0F894B0931D01EBE8F0E0E2
:101240002B9862FF01C02C9A78949FC0B4E095FD62
:1012500007C0F894B0931D012A98299A789495C0F4
:10126000F894B0931D0129982A9A78948EC0B5E01D
:1012700082FF24C095FD11C001E0F894B0931D01D8
:10128000E7E9F0E0009353012C98289862FF02C030
:101290002B9A01C02A9A789478C004E0F894B0930D
:1012A0001D01EBEAF0E0009353012C98289862FFAF
:1012B00002C02D9A01C0299A789467C095FD0BC091
:1012C000F894B0931D01E5E8F0E02C9862FF01C0AE
:1012D0002B9A78945AC0F894B0931D01E1E9F0E09C
:1012E0002C9862FF01C02D9A78944FC0B6E095FD0E
:1012F00007C0F894B0931D012998289A789445C0A6
:10130000F894B0931D012A98289A78943EC0B1E0D1
:1013100082FF24C095FD11C004E0F894B0931D0134
:10132000EBEAF0E0009353012B982A9862FF02C089
:101330002D9A01C0299A789428C001E0F894B093BE
:101340001D01E7E9F0E0009353012D98299862FF11
:1013500002C02B9A01C02A9A789417C095FD0BC041
:10136000F894B0931D01E1E9F0E02B9862FF01C011
:101370002D9A78940AC0F894B0931D01E5E8F0E046
:101380002D9862FF01C02B9A78946F7D089524E810
:1013900030E0F901209253012B982C982D982A982F
:1013A000289829986B7F0895A4E5B1E007E00D9394
:1013B00007E00D9301E00D9304E00D930FEF0D9303
:1013C0000D930BE00D9302E00D9301E00D9301E00E
:1013D0000D93A0E6B1E001E00D9300E00D9304EB66
:1013E0000D930FEF0D930D930D9303E00D930FEFFE
:1013F0000D9301E00D930FEF0D9305E20D9300EDBA
:101400000D9308E70D9308EC0D9304E00D930FEF97
:101410000D9301E00D9300E00D930AE70D9307E0B3
:101420000D9300E00D9301E00D9300E00D930FEF9D
:101430000D93089520915B018B7FB0915C019F7D9E
:10144000B1FD90629F7BB0915D01B1FD906422304F
:1014500011F0886001C0877F08950A95E00FF21DA2
:10146000B4910895E4E5F0E0009154010E942D0A42
:10147000B0937801E4E5F0E0009155010E942D0A57
:10148000B0937901E2E6F0E000915A010E942D0A42
:10149000B0937A0100917301002309F4039501319F
:1014A00008F001E1B02FB00FB00FB09347011B2F30
:1014B000B10FB10FB00FB0934801B10FB00FB00F23
:1014C000B0934901B09170010FEF1CE0B23011F4FC
:1014D00000EA1AE0B33011F402E815E000931201BB
:1014E00010931301E0E7F0E0009177010E942D0ACC
:1014F000B09342010895089520916A0130916B01E3
:10150000B0915C01B33009F43E5097FF02C020E077
:101510003FEFB32FB21B6B2EB25810F4B2E86B2E14
:1015200000E00395609EB12DBD57D8F300934E01A6
:10153000089590680E947C0A0E94450320E030E0F4
:10154000B0E16B2E0E944103B09137012B0F321D89
:101550006A94C1F7B4E036952795BA95E1F7822EE3
:101560009F770E947C0A0895F894E3E0F0E0B9E0E8
:10157000B7BFB491B078C1F3F894A895B4B7B07080
:10158000B4BFB0916000B861B0936000B0E0B093B8
:101590006000B4E0BEBFBFEFBDBF0E94C709B0E0AE
:1015A000B5B9BFE3B4B9B0E0B8B9B0E0B7B9B0E02D
:1015B000BBB9B0E0BAB92224A0E0B0E02D92AA31C4
:1015C000E9F7A0E0B1E00FEF2D920A95E9F7B1E05D
:1015D000B09344010E94D4090E945A0EB0E0B06C4E
:1015E000B0937C00B0917A00B460B068B0937A0098
:1015F00000916C0100934F01B1E0B0930A01F8949F
:101600000E9449030E9454030E9445030E9457030D
:101610000E9445030E945A030E9445030E94F70E50
:101620000E9449030E9449030E944703F8940AEF6D
:101630001AEFA9B196FDA095A2FF1FC01A95C9F790
:101640000A95B1F7E0E0FCE3B591B43E39F4B59109
:10165000B03E21F4B591BF3F09F40CC0E0E0F39532
:10166000F395B591B83F49F4B591B43931F4B591DA
:10167000BA3A19F4EE27F69509940E941A0A0E94C4
:10168000320A0E947B0A0E947C0A00916C0100933E
:101690004F010E94C709B2E0B5BDB2E0B09381002E
:1016A000B2E0B093B100B1E0B5BBB0936E00B2E070
:1016B000B6BBB0936F00B1E0B7BBB0937000B09110
:1016C0007B00BF7BB0937B00B0B7B0917B00B06470
:1016D000B0937B000E943F0378940E944B05B3E0D7
:1016E00096FDB2E0B0936900B1E0BDBBBB27B1602D
:1016F000BCBB8D7F0E944903626033E02CE0B09157
:101700003601BB2321F42CE03A9509F48FCF0E94D7
:10171000450380FF8BCF8E7FB0913701B23070F3DD
:10172000B92FBF710091390100933801B09339018D
:10173000B01721F72A9519F76D7FB3E096FDB2E057
:10174000B0936900BB27B160BCBB8D7FB0917601BF
:10175000BB2321F48062B92FB0709B2F8F7B209226
:1017600007010E94470385FF05C0B0910701BA3009
:1017700008F080640E94410302E085FF01C000E0A0
:10178000B0913701B017B0F3F8940E9454030E944F
:1017900054030E94540378940E9449032092270125
:1017A0000E944103B0916001B13008F48AC0B09149
:1017B0000A01B13008F485C085FD1EC0B091370123
:1017C000BF3F08F47EC0F8940E945D0378940E94A5
:1017D0004703B0913701B130B0F7F8940E94540339
:1017E0000E9443030E94540378940E944703B091DF
:1017F0003701BF3F90F350C3B8E09B2E9068F89438
:101800000E947C0A78940E944703F8949F770E9474
:101810007C0A80903701B0913701BF37789408F483
:1018200058C00E943F03F8940E945D0378949A94F4
:1018300029F70E94990AB82DB550B0936B010E9408
:101840004903F8940E948D0E0E94FD0E7894BAE030
:101850009B2E9068F8940E947C0A78940E9447031B
:10186000F8949F770E947C0A80903701B0913701ED
:10187000BF37789460F70E943F03F8940E945403A6
:101880000E9443030E94540378949A9411F70E9493
:10189000990AB82DBB5FB0936A010E944903F8947E
:1018A0000E948D0E0E941A0F78940E944703F894AC
:1018B0000E947C0A7894B0913701BF3F08F47CCF36
:1018C000EBC200913701B09127010B1710F0009384
:1018D00027010E94470301E0B0915C01B35009F475
:1018E00005E0B0913701B01708F05ACFF8940E9484
:1018F0005D030E945D030E945D0378940E9449038A
:1019000020920A0120920B0120920C01B0910B0150
:10191000B395B0930B01BF3F79F5B0910C01B3952E
:10192000B0930C01B0916E0109E1BA9559F002E350
:10193000BA9541F00DE7BA9529F00AEFBA9511F082
:1019400020920C01B0910C01B017B0F0B0910C01D5
:10195000BA95B0930C01B4EBB0930B01B0916D014B
:10196000B0934F01F8940E945D037894B0916C019C
:10197000B0934F010E9447030E944303B0910801B6
:10198000BB2319F485FF01C051CE01E085FD01C0E4
:1019900006E0B0913701B01708F4B8CF0E944703B2
:1019A000B0910801BB2309F441CEF8940E94C70905
:1019B000209201012092020120920301522C2092D8
:1019C0000401209243017894B0915901BB0FB09368
:1019D000400120921F01209220012092210120929B
:1019E00022012092230120924C0160E070E02092BD
:1019F0001101B8E0B0934C0178600E943F03B0E061
:101A000073FDB0E0B06CB0937C00B0917A00B06828
:101A1000B064B0937A00B0917A00B6FDFCCF00912B
:101A2000780010917900B0917A00BF77B0937A0076
:101A3000112309F00FEF00934D010E94BE05B8E09D
:101A4000B0934C01786080905B01B2E0B0935B0191
:101A50000E941A0A80925B01F894BFEFB0933C0198
:101A60000E943E06B0910101B0933C01B0933D014C
:101A7000B0933E017894B1E0B0930101B0930301BB
:101A80005B2EB0930401B0934601B0913B01B0933B
:101A90004501B0915C01B33019F49F7D87FD9062E0
:101AA0007160726020920D010E9476090E94870980
:101AB0000E9457060E945D060E9457060E945D061E
:101AC0000E94570607C0F8940E941A0A7894209240
:101AD0004C01777F0E94DD070E94D4030E94A30877
:101AE0000E94D6080E945D060E94D60766FD0E94ED
:101AF0004E0476FF0E940A0576FD0E943B050E9477
:101B0000A3080E94E7080E945D060E94DD0766FDAB
:101B10000E9470040E94A3080E9426090E945D068C
:101B20000E94D60766FD0E94AA040E94A3080E9494
:101B300037090E945D060E94DD0766FD0E94DB04F6
:101B40000E94A3080E9476090E945D060E94D607A3
:101B5000B0E073FDB0E0B06CB0937C00B0917A005F
:101B6000B068B064B0937A000E94A3080E9487090D
:101B70000E945D060E94BE0571FF20C067FD1EC069
:101B8000B0913F01B0933C01B0933D01B0913B0156
:101B9000B0934501B1E0B093460118E12CE0B0915B
:101BA0000D01B11728F07D7F746020930F0106C0EE
:101BB000B0913701B13008F08DCF46C072FF10C030
:101BC00067FD0EC0B0910F01BA9511F47B7F7BCFFA
:101BD000B0930F01B0913701B13008F07BCF34C022
:101BE00020921001B0913A01B13058F0B0913F010C
:101BF000B0933D01B0913B01B0934501B1E0B0938A
:101C00004601B0913A010AEFB01708F01DC085FFF8
:101C100004C0B0910801BB23B9F000EF67FF05C015
:101C2000B0913F01B0933C0100E2B0911B01B017AD
:101C300008F450CFB0911001B395B0931001B0915A
:101C40003701BB2309F002C020921001F8940E94D2
:101C5000C70980905B01B2E0B0935B010E941A0A51
:101C600080925B01209201012092020120920301E7
:101C7000522C20920401209240017E7F78940E9491
:101C80003F030E94C709B0E0B06CB0937C00B091F4
:101C90007A00B460B068B0937A0085FF05C0B09157
:101CA0000801BB2309F4C2CCB0916101B13008F046
:101CB00061CD28CEEDE0F0E00E94860E053A09F0F5
:101CC0001EC0EEE0F0E00E94860E0A3509F017C053
:101CD0003AE0A4E5B1E0E3E0F0E00E94860E0D9367
:101CE00031963A95D1F738E1A0E6B1E0EFE0F0E0C7
:101CF0000E94860E0D9331963A95D1F704C00E944A
:101D0000D4090E948D0EE7E2F0E00895F999FECF24
:101D1000E1BDF2BDF89A00B508950E94B00E3AE018
:101D2000A4E5B1E0E3E0F0E00D910E94A80E319649
:101D30003A95D1F738E1A0E6B1E0EFE0F0E00D919F
:101D40000E94A80E31963A95D1F70E94BB0E0895D5
:101D5000F999FECF00BDE1BDF2BDFA9AF99A089556
:101D6000EDE0F0E00FEF0E94A80EEEE0F0E00FEFE4
:101D70000E94A80E0895EDE0F0E005EA0E94A80E8A
:101D8000EEE0F0E00AE50E94A80E089530915001BF
:101D900000915101313011F400935401323011F4AB
:101DA00000935501333011F400935601343011F48F
:101DB00000936801353011F400935701363011F467
:101DC00000935A01373011F400936601383011F452
:101DD00000935B01393011F4009370013A3011F433
:101DE00000935C013B3011F400935D01089525E000
:101DF0000E9449032A95E1F708950E9454030E9426
:101E000057030E945A030E945D030E9443030E94ED
:101E100054030E9457030E945A030E945D030E94CC
:101E200043030E9454030E9457030E945A030E94D6
:101E30005D0308950E945D030E945A030E945703A8
:101E40000E9454030E9443030E945D030E945A03B0
:101E50000E9457030E9454030E9443030E945D03A3
:101E60000E945A030E9457030E94540308958090D1
:101E70005001909051010E9454030E9454030E940B
:101E800054030E9443038A94B1F70E945D030E94A9
:101E900043039A94D1F70895F8940E94FD0E789424
:101EA0000E94F70E0E94F70EB1E0B0935001B1E02E
:101EB000B093510120925201F8940E94370F789408
:101EC000B5E06B2E709037010E944903B091370145
:101ED0007B16C1F7B13018F0BF3F70F10CC00E9403
:101EE000C60EF8940E948D0E0E94FD0EB8E0B093CD
:101EF00060000E94F70E6A9429F7B0915201B395E1
:101F0000B0935201B33008F4D7CF0E94F70EB091CE
:101F10005101B395B0935101F894B0915001BA9525
:101F2000E6E7F0E0EB0FF21D049178940395B09191
:101F30005101B01708F4BECF0E94F70E0E94F70EB1
:101F4000B0915001B395B0935001B0915001BC30A5
:101F500008F4ADCF0E94D409F8940E948D0EB8E029
:0A1F6000B09360000E94F70EFFCA64
:00000001FF
